:1000000000308A00EC2800000A108A100A118207CA
:1000100028340C34013406340A108A100A1182077D
:100020000C345A346B346F34753473346B3461343C
:1000300020347634793470346934733475342E3422
:100040000A34463475346E34673475346A34653432
:10005000213400342330840083130008031941281D
:100060000130F800BF30F7006400F70B3428F80BBC
:1000700032284A30F700F70B3B2800006400800B61
:10008000302800340708F039AA0029080F392A045B
:100090008700061483160610640083120610831668
:1000A000061083120034A708031D5828861059280B
:1000B0008614831686108312A80E2808A9004220F1
:1000C000A80E2808A900422064000C30F700F70BA6
:1000D00067286A2800341430A3002A20F0308316E1
:1000E00087058312861083168610831206108316E6
:1000F00006108312A1012108023C031C872802304C
:10010000A3002A200330A9004220A10A7B28640012
:100110000C30F700F70B8A288D280230A900422006
:1001200064000C30F700F70B93289628A1012108F2
:10013000023C031CA72821080420A200A7012208D2
:10014000A80053200230A3002A20A10A97282E29B4
:1001500001302302A5002408023C031DB1284030D1
:10016000A50725088038A600A7012608A800532067
:10017000003422080C3A0319C728063A0319CF287D
:10018000073A0319D528053A0319DA28DF28A70109
:100190000130A80053200230A3002A20EB280130B0
:1001A000A3000230A400A820EB280130A300A40083
:1001B000A820EB28A7011030A8005320EB28220824
:1001C0001F3C031CE5280730A2050130A7002208C8
:1001D000A8005320EB283829840183131F3083059E
:1001E0000C3083169900A630980090308312980046
:1001F00083161F149F141F159F1107309C00FF309A
:100200008312A00083161F149F141F159F118312C1
:100210001F108316091283129412A012200883164D
:100220008700831220162008831687008312A011EE
:1002300020088316870000308312940083169400F0
:100240000108C73908388100831290010030F80096
:10025000920000308316920083126B286430A30052
:100260002A20A10121080C20A10AF700A200B92828
:0C02700019302102031D32292E296300E1
:02400E00393F38
:00000001FF
